:1000000019C032C031C030C02FC02EC02DC02CC08E
:100010002BC02AC029C028C027C026C025C024C0A4
:1000200023C022C021C020C01FC01FC01DC01CC0D3
:100030001BC01AC011241FBECFEFD2E0DEBFCDBF60
:1000400011E0A0E0B1E0E4EEF7E002C005900D920F
:10005000A631B107D9F711E0A6E1B1E001C01D92C8
:10006000A631B107E1F726C0CBCF1F920F920FB692
:100070000F9211245F9250907900521408F4252CAD
:10008000351408F4352C43945F900F900FBE0F90F9
:100090001F901895CF93C82F8A3011F48DE0FADFA6
:1000A0008091C00085FFFCCFC093C60080E090E047
:1000B000CF910895CFEFD2E0DEBFCDBFCFEF80B7B5
:1000C000806880BF21E023BF599A8DE490E090932F
:1000D000C5008093C40088E08093C1002C2E332497
:1000E000432C569AC7BD82E484BD25BD539A80E84F
:1000F0008093B40081E28093B0002093B10080E649
:1001000080937C008FEB80937A008FEE80937A004F
:1001100020937E00229A2A9A789488954420E9F7C1
:10012000F8948FEB80937A00832D82198093B4002A
:100130008091B4009FEF292E33241A9A99279F9318
:100140008F938C2F992701969F938F938EE091E048
:100150009F938F9380E091E09F938F930FD0C15036
:10016000C7BD8FEE80937A0078948DB79EB70896BE
:100170000FB6F8949EBF0FBE8DBFCFCFA0E0B0E00A
:10018000E3ECF0E008C38F819885AE01475F5F4FD5
:10019000BC018D819E8102D0E2E019C3A2E1B0E0F2
:1001A000E3EDF0E0E8C2EE24FF2487011C017E8726
:1001B0006D872A01CC24DD24FC01D782C68283818D
:1001C00081FD55C28FEF9FEF65C28D859E8501969B
:1001D0009E878D87C0FE39C28F8580538A30D0F4C8
:1001E0009F85903339F4662029F4C3FC03C0E0E016
:1001F000F1E08DC08AE0689E602C1124FF856F0EAF
:1002000020ED620E67FE02C05FE7652EC3FC2FC2C1
:10021000762C2DC2C3FE04C0662011F441E0642E8A
:10022000EF858E2F992787FD9095883691058CF55F
:10023000853691050CF06EC08335910509F492C0A6
:1002400084359105CCF48B32910509F449C08C3288
:1002500091054CF48032910509F446C08332910532
:1002600009F44AC0EDC18D32910509F440C08E32C7
:10027000910509F444C0E4C18336910509F450C0E6
:10028000843691050CF087C08835910509F4B9C012
:10029000D7C18037910509F4AEC08137910584F448
:1002A0008C36910591F18D3691052CF489369105A6
:1002B00009F471C0C5C18F36910509F499C0C0C158
:1002C0008537910509F49FC08637910524F483375B
:1002D000910571F1B5C18837910509F492C0B0C19B
:1002E00080E190E0C82AD92AE0E2F0E010C080E87E
:1002F00090E0C82AD92ABBC1E0E4F0E008C088E059
:1003000090E0C82AD92A6624B2C1E4E0F0E0CE2AFF
:10031000DF2AADC13FE3E32E7A94F3E6FF8731C1D4
:10032000F20182E090E0480E591EE0807A9429C1E3
:10033000F20182E090E0480E591EA081B1817D015A
:10034000C3FE08C0862D992787FD9095BC01CD017D
:10035000B8D11DC0FD0101900020E9F73197EA1BDB
:10036000E88B16C0F20182E090E0480E591E019021
:10037000F081E02D7F01C3FE08C0862D992787FDFF
:100380009095BC01CF0192D102C0CF0186D1888B5C
:100390009889791AF6C0C2FE0AC0F20184E090E0A2
:1003A000480E591E20813181428153810CC0F201D7
:1003B00082E090E0480E591E808191819C01442783
:1003C00037FD4095542F79018A0157FF0CC0E2E0B8
:1003D000F0E0CE2ADF2A10950095F094E094E11C1D
:1003E000F11C011D111D8FEB9FEFC822D92227C0E0
:1003F00098E0988B08C0E0E4F0E0CE2ADF2AF8E726
:10040000FF8720E1288BC2FE0AC0F20184E090E061
:10041000480E591E20813181428153810AC0F20168
:1004200082E090E0480E591E808191819C01442712
:10043000552779018A01EFECFFEFCE22DF22CE01B2
:1004400001969A8B898B9889892E9924AA24BB249A
:10045000C801B701A50194016CD1DC01CB01E98988
:10046000FA8980838A3024F0FF858F0F815201C082
:10047000805DE989FA898193FA8BE98BC801B7011C
:10048000A501940156D179018A0121153105410553
:100490005105F1F6E98881E090E08C0F9D1FE81A84
:1004A000C60182739070892B09F07A94C6FE0DC044
:1004B000872D992787FD9095E889E03121F42EEF6B
:1004C000722E780E02C0782E7A94C3FE0FC0262DAD
:1004D000332727FD30958E2D9927821793072CF00F
:1004E00087EF9FEFC822D92201C06E18C3FE02C059
:1004F000761801C07E18C60180789170892B49F466
:10050000872D7A9418162CF4B10180E290E0E4D0A3
:10051000F7CFC1FE04C0B1018DE290E00BC0C4FE74
:1005200004C0B1018BE290E005C0C5FE04C0B1017A
:1005300080E290E0D1D0C6FE0EC0B10180E390E031
:10054000CBD09889903139F4B101EF858E2F99275E
:1005500087FD9095C1D0D0FE09C0872D7A941816DA
:100560002CF4B10180E390E0B7D0F7CFC3FE09C00F
:10057000862D6A9418162CF4B10180E390E0ACD07B
:10058000F7CF90E8B92EBC2049F4872D7A9418163D
:100590002CF4B10180E290E09FD0F7CFFF85F336D5
:1005A00039F48E2DB101992787FD909595D03DC0E6
:1005B0002F852337A9F488898150888B8F3FA9F133
:1005C000F70180810894E11CF11CB101992787FD96
:1005D000909582D098899150988B9F3F89F725C03C
:1005E000EF85E33571F4F889F150F88BFF3FE9F0BE
:1005F000F7018491B10199276FD00894E11CF11C97
:10060000F2CF6E010894C11CD11C89899A898C157E
:100610009D0559F0E989FA898291FA8BE98BB1013C
:10062000992787FD909558D0F0CFBB2059F0872DA2
:100630007A9418163CF4B10180E290E04DD0F7CFE7
:10064000B1014AD0CC24DD2412C09F85953241F4FB
:1006500081E0C82ED12C6624762CEAE0E88B07C016
:10066000B101FF858F2F992787FD909535D0F10136
:10067000838183FF04C0ED85FE85F49103C0ED8581
:10068000FE85F081FF872F85222309F09ECDF101A1
:1006900086819781E2E162968AC0FC010590002084
:1006A000E9F7809590958E0F9F1F0895FC010590A6
:1006B000615070400110D8F7809590958E0F9F1F64
:1006C0000895FC016150704001900110D8F78095A9
:1006D00090958E0F9F1F08950F931F93CF93DF93D5
:1006E0008C01EB018B81992781FF1CC082FF0DC01B
:1006F0002E813F818C819D812817390764F4E88120
:10070000F9810193F983E88306C0E885F985802F94
:100710000995892B39F48E819F8101969F838E8361
:10072000C80102C08FEF9FEFDF91CF911F910F9112
:100730000895A1E21A2EAA1BBB1BFD010DC0AA1F22
:10074000BB1FEE1FFF1FA217B307E407F50720F03A
:10075000A21BB30BE40BF50B661F771F881F991FB5
:100760001A9469F760957095809590959B01AC01FE
:10077000BD01CF0108952F923F924F925F926F92E9
:100780007F928F929F92AF92BF92CF92DF92EF9221
:10079000FF920F931F93CF93DF93CDB7DEB7CA1BA2
:1007A000DB0B0FB6F894DEBF0FBECDBF09942A88CD
:1007B000398848885F846E847D848C849B84AA8475
:1007C000B984C884DF80EE80FD800C811B81AA8102
:1007D000B981CE0FD11D0FB6F894DEBF0FBECDBFCD
:0407E000ED0108958A
:1007E40000000002000000004A0000000000256430
:0607F4002025640A00004C
:00000001FF
